:1000000000308A00892900000A108A100A1182072C
:1000100028340C34013406340A108A100A1182077D
:1000200076347934733469346C3461346D3400342B
:100030002F308400000803192C280130A100A001F2
:10004000A00B2028A10B1F284A30A000A00B2628B7
:1000500000000000800B1D28003406080F39B50091
:10006000340EA000F030A0052008F03935048600D9
:100070000615831606110000831206118316061159
:1000800083120034B208031D4728861048288614BE
:10009000831686108312B30E3308B4002D20B30EDE
:1000A0003308B4002D200D30A000A00B55280034DB
:1000B0001430AF0018200F30831686058312861087
:1000C0008316861083120611831606118312AB0164
:1000D0002B08023C031C74280230AF0018200330A8
:1000E000B4002D20AB0A68280D30A000A00B7628A4
:1000F0000230B4002D200D30A000A00B7D28AB01F4
:100100002B08023C031C90282B080420AC00B201F1
:100110002C08B30042200230AF001820AB0A802820
:100120008A11CB2901302E02B0002F08023C031D9A
:100130009B284030B00730088038B100B201310848
:10014000B300422000342D08A0000C302002031917
:10015000B6280A3020020319BE280D3020020319E8
:10016000C428083020020319C928CE28B201013062
:10017000B30042200230AF001820DA280130AE0070
:100180000230AF009220DA280130AE00AF0092209A
:10019000DA28B2011030B3004220DA282D081F3CC3
:1001A000031CD4280730AD050130B2002D08B30080
:1001B0004220DA2800342E08A1012D020318E3287A
:1001C0002D08A000EF28A0010830AF00AD0DA00D54
:1001D0002E0820020318A000A10DAF0BE628003462
:1001E0002B08A000AB1BF8282C1D02292030FD286D
:1001F000A009A00A2008AB002D30A100AD00A3206B
:100200002C1DAC152B08AD006430AE00DB2020089F
:10021000AB0021083030031D14292C18AC15AC1983
:100220001A292C1A20301629AC112C12A1072108EA
:10023000AD00A3202B08AD000A30AE00DB20200863
:10024000AB0021083030031D2929AC192D292C1AA7
:100250002030A1072108AD00A3203030AB072B08C8
:10026000AD00A3200034A91129088316870083124A
:1002700087155330A000A00B3B29A911290883162C
:100280008700831287115330A000A00B452900344A
:100290000130AF0018203321AE012E08033C031CAF
:1002A00075292D08A0002E08A10003195B29031051
:1002B000A00CA10B5729201C7229A911290883160B
:1002C0008700831287115330A000A00B6529A91164
:1002D000290883168700831287155330A000A00BCE
:1002E0006F2973293321AE0A4D29A91129088316D4
:1002F00087008312871100340F30AD0048212C088D
:10030000AD0048212B08AD0048212B08AD00482145
:10031000003484011F308305073083169F00FF30AF
:100320008312A900AA01043083169F0083121F08BC
:10033000383901389F009412A912290883168700C2
:10034000831229162908831687008312A911290808
:100350008316870000308312940083169400831262
:10036000A001A01DBB290730810181308400000855
:10037000C0390F3880006400813084000008C03923
:100380002004800090010030A1009200003083160C
:100390009200831258280C30AD00A3200730AE0025
:1003A0000230AF009220AB012B080C20AB0AAD004D
:1003B000A32007302B02031DD4290030A1001F0801
:1003C000C73921049F000130AE00AF0092201F15F5
:1003D0001F19E8291E081E0EA7000F30A705583068
:1003E000AD00A3203A30AD00A3202030AD00A32003
:1003F0002708AB001830AC00F0200630AB002030EE
:10040000AD00A320AB0BFF290830A1001F08C7399E
:1004100021049F000130AE000230AF0092201F1572
:100420001F19102A1E081E0EA8000F30A8055930EB
:10043000AD00A3203A30AD00A3202030AD00A320B2
:100440002808AB001830AC00F0200630AB0020309C
:10045000AD00A320AB0B272A2708AB000130AC006E
:100460007C212808AB000230AC007C21291329082C
:0C0470008316870083120713DD29630048
:02400E00F13F80
:00000001FF
